:020000040000FA
:06000000A1EF1AF012004E
:060008006FEF14F012007E
:06002A0002007934000021
:10003000FD000000010000006E350000000000001F
:0400400018000000A4
:0C0044000001EA6BEB6B8A6A896AF90E16
:10005000926E010EC26E0E0EC16E860EC06EBA6A30
:10006000BD6A010E066E640EEC6FD00EEF6F070EC8
:10007000F06F080EED6F0B0EEE6F000E036E046A4C
:10008000096E0A6A076E086A800ED56E1200F2A425
:1000900018D0F2940001EB2B050E0101005D07E280
:1000A0000A0E0001EB5D03E38974EB6B1200050E91
:1000B0000101005D06E12E0E0001EB5D02E3897493
:1000C000EB6B1200E4DF050E0101005D45E36D50AE
:1000D000020B01E012000001EA5129E0800E040148
:1000E0000C1525E1400EE66E600EE66E000EE66E23
:1000F00006EC15F0E552E552E5520001EA6B016AA3
:100100000250015C13E20150EA6AE00FE96E000E52
:10011000EA22EF50E66E0150EA6A600FE96E000EC7
:10012000EA22E552E750EF6E012AEAD7026A00019F
:10013000FD51005C10E3400EE66EA00EE66E000E70
:10014000E66E48EC15F0E552E552E5520001FD6F10
:10015000E85001E0006A01D81200D9CFE6FFE1CFF4
:10016000D9FF090EE1260001FD51005C02E32FEFEB
:1001700014F00001EA5102E02FEF14F089820050E0
:10018000EA6AA00FE96E000EEA22EF50F10A02E1DE
:10019000E2EF13F0010A02E1A5EF13F0020A02E117
:1001A00088EF13F0CF0A02E13DEF13F0010A02E1FC
:1001B000F9EF12F0070A02E1F0EF12F0010A02E192
:1001C000A7EF12F0030A02E159EF12F0010A02E16F
:1001D00048EF12F00F0A02E11FEF12F0010A02E1EC
:1001E000D2EF11F0030A02E175EF11F0010A02E10A
:1001F00006EF11F0070A02E18BEF10F0010A02E1AD
:1002000052EF10F0030A02E119EF10F0010A02E1C7
:10021000DCEF0FF01F0A02E187EF0FF0020A02E1A4
:10022000EFEF0EF0030A02E127EF0EF0020A02E1FF
:100230004EEF0DF0070A02E1F2EF0CF0010A02E1C5
:100240009FEF0CF0030A02E14EEF0CF0010A02E10D
:10025000CDEF0BF00F0A02E14DEF0BF0010A02E1C6
:10026000F2EF0AF0030A02E1ABEF0AF0010A02E141
:1002700045EF0AF0070A02E10FEF0AF0010A02E176
:10028000D9EF09F0030A02E193EF09F0010A02E154
:1002900012EF08F03F0A02E1E1EF07F0010A02E184
:1002A000C7EF07F0030A02E1ABEF07F0010A02E132
:1002B00091EF07F0070A02E175EF07F0010A02E18A
:1002C00057EF07F0030A02E13BEF07F0010A02E1F2
:1002D00021EF07F00F0A02E1D8EF06F0010A02E170
:1002E000BFEF06F0030A02E175EF06F0010A02E132
:1002F0002DEF06F0070A02E1D0EF05F0010A01E157
:10030000F1D3030A01E194D3010A01E178D31F0A72
:1003100001E1F9D2010A01E1AAD2030A01E11DD2E9
:10032000010A01E1F9D1070A01E1C7D1010A01E19E
:10033000ACD1030A01E193D1010A01E17AD10F0A9C
:1003400001E1F9D0010A01E1EAD0030A01E1C1D0DB
:10035000010A01E19BD0070A67E0010A43E0030AB2
:100360000AE0010A02E028EF14F0E66A3AEC14F021
:10037000E5522DEF14F0010EE66E3AEC14F0E55262
:1003800061DEE66A3AEC14F0E552060EE66E3AECEF
:1003900014F0E552010EE66E3AEC14F0E552E66A0E
:1003A0003AEC14F0E552E66A3AEC14F0E552010E2C
:1003B000E66E3AEC14F0E552200EE66E3AEC14F0DC
:1003C000E552520EE66E3AEC14F0E552530EE66E2C
:1003D0003AEC14F0E552540EE66E3AEC14F0E552A5
:1003E0002DEF14F0020EE66E3AEC14F0E552E66AD8
:1003F0003AEC14F0E552060EE66E3AEC14F0E552D3
:10040000010EE66E3AEC14F0E552E66A3AEC14F0AE
:10041000E552E66A3AEC14F0E552010EE66E3AEC6B
:1004200014F0E5522DEF14F0030EE66E3AEC14F0E2
:10043000E5520028186E0001FD51185C18E2002AF0
:100440000050EA6AA00FE96E000EEA22EFCFDFFF4C
:100450003D0EDF5C06E2DFCFE6FF3AEC14F0E5523A
:1004600005D0FE0EE66E3AEC14F0E5520DD0FE0E0D
:10047000E66E3AEC14F0E5520028EA6AA00FE96E45
:10048000000EEA22040EEF6E2DEF14F0400E015C18
:1004900009E20150EA6A600FE96E000EEA22EF6A93
:1004A000012AF4D7016A04010CBF0CD0400EE66E9D
:1004B000600EE66E000EE66E06EC15F0E552E552B3
:1004C000E55203D00001010EEA6FFDC000F02DEFF0
:1004D00014F0050EE66E3AEC14F0E552000E036ED1
:1004E000046A096E0A6A076E086A840ECB6E040EEF
:1004F000CA6E0B0EBC6EB80EBB6E9E9C9D8CB36A12
:10050000B26A890EB16E0B0EBA6EBE6A0C0EBD6E6B
:100510009494C00EF26E1E0ED26E2DEF14F0060EE5
:10052000E66E3AEC14F0E5529D9CBA6ABD6A0E0E76
:10053000D26E2DEF14F0070EE66E3AEC14F0E55291
:10054000030E0024186E0001FD51185C63E2002ABE
:100550000050EA6AA00FE96E000EEA22EF500D6E1D
:100560000D50030A40E0010A2BE0030A16E0010ADD
:1005700001E04CD0002A0050EA6AA00FE96E000E9C
:10058000EA22EF50066E002A0050EA6AA00FE96ED8
:10059000000EEA22EFCFECF03CD0002A0050EA6ACD
:1005A000A00FE96E000EEA22EFCFF0F0002A005013
:1005B000EA6AA00FE96E000EEA22EFCFEFF029D031
:1005C000002A0050EA6AA00FE96E000EEA22EFCF7F
:1005D000F2F0002A0050EA6AA00FE96E000EEA224B
:1005E000EFCFF1F016D0002A0050EA6AA00FE96EB2
:1005F000000EEA22EFCFEDF0002A0050EA6AA00FC9
:10060000E96E000EEA22EFCFEEF003D0020E0026D4
:1006100000D00DD0FE0EE66E3AEC14F0E552002844
:10062000EA6AA00FE96E000EEA22040EEF6E2DEFCB
:1006300014F0080EE66E3AEC14F0E552F29E065005
:100640000D6E0D5009E000000000000000000000E9
:10065000000000000D06F5D7F28E2DEF14F0090E04
:10066000E66E3AEC14F0E552F29EECC00DF00D503F
:1006700009E0000000000000000000000000000091
:100680000D06F5D7F28E2DEF14F00A0EE66E3AEC59
:1006900014F0E552F29EEFC013F0F0C014F01350C6
:1006A000141008E000000000000000001306000E17
:1006B000145AF5D7F28E2DEF14F00B0EE66E3AECCD
:1006C00014F0E5520028186E0001FD51185C15E287
:1006D000002A0050EA6AA00FE96E000EEA22EF50ED
:1006E0000D6E0D5009E00000000000000000000049
:1006F000000000000D06F5D70DD0FE0EE66E3AECB8
:1007000014F0E5520028EA6AA00FE96E000EEA2212
:10071000040EEF6E2DEF14F0A1940C0EE66E3AEC81
:1007200014F0E552C282C2B2FED7A1A40AD0E66A92
:100730003AEC14F0E552E66A3AEC14F0E5522DEF8B
:1007400014F0C450E66E3AEC14F0E552C350E66E75
:100750003AEC14F0E5522DEF14F00D0EE66E3AEC83
:1007600014F0E5520028186E0001FD51185C70E28B
:100770009D50400B03E0D250200B06E1FE0EE66ECA
:100780003AEC14F0E55263D0A194002A0050EA6AD2
:10079000A00FE96E000EEA22EF50136E146A13C028
:1007A0000BF014C00CF0070E0C02F3CF0CF0070E88
:1007B0000B02F3CF0BF0F4500C260F0E0D6EE80E6B
:1007C000136E030E146E1350141008E000000000A6
:1007D000000000001306000E145AF5D70D06083469
:1007E00004E207500E08000E085408E3D8800850B1
:1007F00004E7F20E075CFF0E085802E20D50DFE13D
:10080000A1A405D0E66A3AEC14F0E55220D00834F1
:1008100004E207500E08000E085408E3D880085080
:1008200004E7F20E075CFF0E085806E2FE0EE66EC5
:100830003AEC14F0E5520BD00050EA6AA00FE96ED2
:10084000000EEA22EF50E66E3AEC14F0E5520DD0BD
:10085000FE0EE66E3AEC14F0E5520028EA6AA00FAC
:10086000E96E000EEA22040EEF6E2DEF14F00E0E6C
:10087000E66E3AEC14F0E5520028186E0001FD51C6
:10088000185C32E2002A0050EA6AA00FE96E000EFE
:10089000EA22EF500D6E010E0D1402E0000E01D0A1
:1008A000010EE8B08B82E8A08B92020E0D1402E0DC
:1008B000010E01D0000EE8B09482E8A09492040EDC
:1008C0000D1402E0010E01D0000EE8B08B80E8A00C
:1008D0008B90080E0D1402E0010E01D0000EE8B05E
:1008E0009480E8A094900DD0FE0EE66E3AEC14F0E1
:1008F000E5520028EA6AA00FE96E000EEA22040E13
:10090000EF6E2DEF14F00F0EE66E3AEC14F0E55298
:100910000028186E0001FD51185C62E2002A0050A8
:10092000EA6AA00FE96E000EEA22EF50010B02E026
:10093000010E01D0000EE8B08A8AE8A08A9A005021
:10094000EA6AA00FE96E000EEA22EF50020B02E005
:10095000010E01D0000EE8B0938AE8A0939A0050EF
:10096000EA6AA00FE96E000EEA22EF50040B02E0E3
:10097000010E01D0000EE8B08A8CE8A08A9C0050DD
:10098000EA6AA00FE96E000EEA22EF50080B02E0BF
:10099000010E01D0000EE8B0938CE8A0939C0050AB
:1009A000EA6AA00FE96E000EEA22EF50100B02E097
:1009B000010E01D0000EE8B08A8EE8A08A9E005099
:1009C000EA6AA00FE96E000EEA22EF50200B02E067
:1009D000010E01D0000EE8B0938EE8A0939E0DD0DA
:1009E000FE0EE66E3AEC14F0E5520028EA6AA00F1B
:1009F000E96E000EEA22040EEF6E2DEF14F0100ED9
:100A0000E66E3AEC14F0E5520D6A8ABA0D8093BA9C
:100A10000D828ABC0D8493BC0D868ABE0D8893BE60
:100A20000D8A0D50E66E3AEC14F0E5522DEF14F0FD
:100A3000110EE66E3AEC14F0E552020E0024186E28
:100A40000001FD51185C3FE2002A0050EA6AA00F45
:100A5000E96E000EEA22EFCF14F0002A0050EA6A95
:100A6000A00FE96E000EEA22EFCF13F0F29E8A9AF1
:100A70008A8C8A9C8A8C8A9C8A8C8A9C8A8C8A9C86
:100A80008A8C8A9C8A8C8A9C06500D6E0D5009E0D7
:100A900000000000000000000000000000000D0643
:100AA000F5D78A8C8A9C0E0E0D6E14321332819A01
:100AB000D8B0818A818C819C0D2EF7D78A9A8A8C36
:100AC0008A9CF28E0DD0FE0EE66E3AEC14F0E552E2
:100AD0000028EA6AA00FE96E000EEA22040EEF6E0B
:100AE0002DEF14F0120EE66E3AEC14F0E552020E01
:100AF0000024186E0001FD51185C43E2002A0050EA
:100B0000EA6AA00FE96E000EEA22EFCF14F0002A85
:100B10000050EA6AA00FE96E000EEA22EFCF13F050
:100B2000F29E8A9A8A8C8A9C00008A8A8A8C8A9C85
:100B300000008A9A8A8C8A9C8A8C8A9C8A8C8A9CDD
:100B40008A8C8A9C06500D6E0D5009E00000000052
:100B5000000000000000000000000D06F5D78A8CA0
:100B60008A9C0E0E0D6E14321332819AD8B0818A8F
:100B7000818C819C0D2EF7D78A9A8A8C8A9CF28E62
:100B80000DD0FE0EE66E3AEC14F0E5520028EA6A4B
:100B9000A00FE96E000EEA22040EEF6E2DEF14F0A6
:100BA000130EE66E3AEC14F0E5520028186E0001C0
:100BB000FD51185C43E2002A0050EA6AA00FE96E7A
:100BC000000EEA22EFCF13F0F29E8A8A8A8C8A9C6A
:100BD0008A8C8A9C00008A9A8A8C8A9C8A8C8A9C3D
:100BE0008A8C8A9C8A8C8A9C06500D6E0D5009E076
:100BF00000000000000000000000000000000D06E2
:100C0000F5D78A8C8A9C080E0D6E1332819AD8B063
:100C1000818A818C819C0D2EF8D78A9A8A8C8A9C35
:100C20008A8C8A9C8A8C8A9C8A8C8A9C8A8C8A9CD4
:100C30008A8C8A9C8A8C8A9CF28E0DD0FE0EE66E7F
:100C40003AEC14F0E5520028EA6AA00FE96E000EB3
:100C5000EA22040EEF6E2DEF14F0140EE66E3AEC5D
:100C600014F0E552F29E8A9A8A8C8A9C8A8C8A9C1D
:100C700000008A8A8A8C8A9C00008A9A8A8C8A9CC4
:100C80008A8C8A9C8A8C8A9C938A06500D6E0D50A1
:100C900009E000000000000000000000000000006B
:100CA0000D06F5D78A8C8A9C0E0E0D6E8A8C8A9C56
:100CB000D89081BAD880143213320D2EF7D7D8903D
:100CC00014321332D890143213328A8C939A8A9C3D
:100CD000F28E14C0E6FF3AEC14F0E55213C0E6FFC2
:100CE0003AEC14F0E5522DEF14F0150EE66E3AECE6
:100CF00014F0E552F29E8A8A8A8C8A9C00008A9AB5
:100D00008A8C8A9C00008A8A8A8C8A9C00008A9A33
:100D10008A8C8A9C8A8C8A9C8A8C8A9C938A0650AC
:100D20000D6E0D5009E00000000000000000000002
:100D3000000000000D06F5D78A8C8A9C080E0D6E07
:100D40008A8C8A9CD89081BAD88013320D2EF8D71D
:100D50008A8C8A9C8A8C8A9C8A8C8A9C8A8C8A9CA3
:100D60008A8C8A9C8A8C8A9C8A8C939A8A9CF28E22
:100D700013C0E6FF3AEC14F0E5522DEF14F0160E16
:100D8000E66E3AEC14F0E552F29E8A9A8A8C8A9CBE
:100D900000008A8A8A8C8A9C8A8C8A9C8A9A8A8C8D
:100DA0008A9C8A8C8A9C8A8C8A9CF28E2DEF14F005
:100DB000170EE66E3AEC14F0E5520028186E0001AA
:100DC000FD51185C2FE2F29E002A0050EA6AA00F43
:100DD000E96E000EEA22EFCF13F00001135020E07D
:100DE0008A9A8A8C8A9C00008A8A8A8C8A9C8A8C3D
:100DF0008A9C8A9A8A8C8A9C8A8C8A9C8A8C8A9CF5
:100E000006500D6E0D5009E00000000000000000CB
:100E10000000000000000D06F5D700011306DDD725
:100E2000F28E0DD0FE0EE66E3AEC14F0E55200287C
:100E3000EA6AA00FE96E000EEA22040EEF6E2DEFB3
:100E400014F0180EE66E3AEC14F0E552F29E8A9A0F
:100E50008A8C8A9C8A8C8A9C8A8C8A9C00008A8ACA
:100E60008A8C8A9C00008A9A8A8C8A9C8A8C8A9CAA
:100E7000F28E2DEF14F0190EE66E3AEC14F0E552F6
:100E8000F29E8A8A8A8C8A9C00008A9A8A8C8A9C22
:100E90008A8C8A9C00008A8A8A8C8A9C00008A9AA2
:100EA0008A8C8A9C8A8C8A9CF28E2DEF14F01A0E02
:100EB000E66E3AEC14F0E552F29E8A9A8A8C8A9C8D
:100EC00000008A8A8A8C8A9C00008A9A8A8C8A9C72
:100ED00000008A8A8A8C8A9C00008A9A8A8C8A9C62
:100EE0008A8C8A9CF28E2DEF14F01B0EE66E3AEC83
:100EF00014F0E552F29E8A8A8A8C8A9C8A8C8A9C9B
:100F000000008A9A8A8C8A9C00008A8A8A8C8A9C31
:100F100000008A9A8A8C8A9C8A8C8A9CF28E2DEF99
:100F200014F01C0EE66E3AEC14F0E552F29E8A9A2A
:100F30008A8C8A9C00008A8A8A8C8A9C8A8C8A9CE9
:100F40008A8C8A9C00008A9A8A8C8A9C8A8C8A9CC9
:100F5000F28E2DEF14F01D0EE66E3AEC14F0E55211
:100F6000F29E8A8A8A8C8A9C00008A9A8A8C8A9C41
:100F70008A8C8A9C8A8C8A9C00008A8A8A8C8A9CA9
:100F800000008A9A8A8C8A9CF28E2DEF14F01E0E35
:100F9000E66E3AEC14F0E552F29E8A9A8A8C8A9CAC
:100FA0008A8C8A9C8A8C8A9C00008A8A8A8C8A9C79
:100FB0008A8C8A9C00008A9A8A8C8A9CF28E2DEFF9
:100FC00014F01F0EE66E3AEC14F0E5520028186E8D
:100FD0000001FD51185C17E2002A0050EA6AA00FD8
:100FE000E96E000EEA22EFCF13F0F29E060E0D6EB0
:100FF0001332819AD8B0818A818C819C0D2EF8D7CA
:101000008A9AF28E0DD0FE0EE66E3AEC14F0E5529E
:101010000028EA6AA00FE96E000EEA22040EEF6EC5
:101020002DEF14F0200EE66E3AEC14F0E552020EAD
:101030000024186E0001FD51185C01E365D1002AFF
:101040000050EA6AA00FE96E000EEA22EFCF14F01A
:10105000002A0050EA6AA00FE96E000EEA22EFCFE4
:1010600013F0010E13C0DBFF020E14C0DBFFF29E73
:101070008A9A8A8C8A9C00008A8A8A8C8A9C0000C0
:101080008A9A8A8C8A9C8A8C8A9C8A8C8A9C8A8C72
:101090008A9C06500D6E0D5009E000000000000013
:1010A00000000000000000000D06F5D78A8C8A9C25
:1010B0000E0E0D6E14321332819AD8B0818A818C53
:1010C000819C0D2EF7D78A9A8A8C8A9C030EDB6A44
:1010D000040EDB6A030EDBCF18F0040EDBCF19F031
:1010E0000001ED51000119AE02D0D89003D0185C78
:1010F000000E195801E397D08A9A8A8C8A9C8A8CB0
:101100008A9C8A8C8A9C00008A8A8A8C8A9C00002D
:101110008A9A8A8C8A9C8A8C8A9CECC00DF00D502D
:1011200009E00000000000000000000000000000D6
:101130000D06F5D78A9A8A8C8A9C00008A8A8A8C46
:101140008A9C8A8C8A9C8A8C8A9C00008A9A8A8CC7
:101150008A9C8A8C8A9C06500D6E0D5009E0000016
:101160000000000000000000000000000D06F5D7A0
:101170008A9A8A8C8A9C8A8C8A9C00008A8A8A8CA9
:101180008A9C00008A9A8A8C8A9C8A8C8A9C8A8C87
:101190008A9C938A06500D6E0D5009E000000000F5
:1011A000000000000000000000000D06F5D78A8C4A
:1011B0008A9C0E0E0D6E8A8C8A9CD89081BAD8803B
:1011C000143213320D2EF7D7D89014321332D89030
:1011D000143213328A8C939A8A9C06500D6E0D50ED
:1011E00009E0000000000000000000000000000016
:1011F0000D06F5D7010EDBCF18F0020EDBCF19F08C
:101200001350181802E11450191807E1030EDB50AF
:101210000D6E030EDB68040EDB6A030EDB2A040E80
:1012200001E3DB2A57D7F28EF29ED950030FE96E05
:10123000DACFEAFFFF0EEE1801E1ED505EE10D504E
:10124000E66E3AEC14F0E5520001EE510D02F35057
:10125000E66ED950030FE96EDACFEAFFE552E750A8
:10126000EE6EED6AD950030FE96EDACFEAFFEE5069
:10127000ED1042E08A9A8A8C8A9C8A8C8A9C8A8C9D
:101280008A9C00008A8A8A8C8A9C00008A9A8A8CAE
:101290008A9C8A8C8A9CECC00DF00D5009E00000FD
:1012A0000000000000000000000000000D06F5D75F
:1012B0008A9A8A8C8A9C00008A8A8A8C8A9C8A8C68
:1012C0008A9C8A8C8A9C00008A9A8A8C8A9C8A8C46
:1012D0008A9C06500D6E0D5009E0000000000000D1
:1012E00000000000000000000D06F5D7030EDB062D
:1012F000040E01E2DB06B6D705D0FE0EE66E3AEC30
:1013000014F0E552F28E0DD0FE0EE66E3AEC14F0BB
:10131000E5520028EA6AA00FE96E000EEA22040EE8
:10132000EF6E2DEF14F0210EE66E3AEC14F0E5525C
:10133000020E0024186E0001FD51185C2BE2F29E93
:101340008A8C939A8A9A8A9C8A8C8A9C8A8C8A9C98
:101350008A8C8A9C002A0050EA6AA00FE96E000E6F
:10136000EA22EFCF14F0002A0050EA6AA00FE96EDB
:10137000000EEA22EFCF13F0100E0D6E143213326E
:10138000819AD8B0818A818C819C0D2EF7D78A9A58
:10139000F28E0DD0FE0EE66E3AEC14F0E552002807
:1013A000EA6AA00FE96E000EEA22040EEF6E2DEF3E
:1013B00014F0220EE66E3AEC14F0E552F29E8A8C9E
:1013C000939A8A9A8A9C8A8A8A8C8A9C8A9A8A8C1C
:1013D0008A9C8A8C8A9C8A8C8A9C8A8C8A9C8A8C1D
:1013E0008A9C8A8C8A9C8A8C8A9C8A8C8A9C8A8C0D
:1013F0008A9C8A8C8A9C938A080E0D6E818C819CB3
:10140000D89081BAD88013320D2EF8D78A9AF28EEE
:1014100013C0E6FF3AEC14F0E5522DEF14F0230E62
:10142000E66E3AEC14F0E552F29E8A8C939A8A9A10
:101430008A9C8A8C8A9C8A8C8A9C8A8A8A8C8A9CBE
:101440008A9A8A8C8A9C8A8C8A9C8A8C8A9C8A8CAE
:101450008A9C8A8C8A9C8A8C8A9C8A8C8A9C8A8C9C
:101460008A9C938A080E0D6E818C819CD89081BADB
:10147000D88013320D2EF8D78A9AF28E13C0E6FF69
:101480003AEC14F0E5522DEF14F0240EE66E3AEC2F
:1014900014F0E552002A0050EA6AA00FE96E000E2F
:1014A000EA22EF500D6E0001FD51005C45E2015053
:1014B0000D24186E400E185C3FE20D50E66E3AECBB
:1014C00014F0E552050E0DC0DBFF050EDB5033E0D6
:1014D000F29E8A8C939A8A8A8A9C8A9A8A8C8A9C9F
:1014E0008A8C8A9C8A8A8A8C8A9C8A9A8A8C8A9C10
:1014F0008A8C8A9C8A8C8A9C8A8C8A9C8A8C8A9CFC
:101500008A8C8A9C8A8C8A9C8A8C8A9C938A080EF4
:101510000D6E818C819CD89081BAD88013320D2EAB
:10152000F8D78A9AF28E13C0E6FF3AEC14F0E5522F
:10153000050EDB06CAD70DD0FE0EE66E3AEC14F0AF
:10154000E5520028EA6AA00FE96E000EEA22040EB6
:10155000EF6E2DEF14F0250EE66E3AEC14F0E55226
:10156000020E0024186E0001FD51185C2CE2F29E60
:101570008A8C939A8A9A8A9C8A8C8A9C8A8A8A8C78
:101580008A9C8A8C8A9C002A0050EA6AA00FE96E25
:10159000000EEA22EFCF14F0002A0050EA6AA00FF2
:1015A000E96E000EEA22EFCF13F0100E0D6E14322A
:1015B0001332819AD8B0818A818C819C0D2EF7D705
:1015C0008A9AF28E0DD0FE0EE66E3AEC14F0E552D9
:1015D0000028EA6AA00FE96E000EEA22040EEF6E00
:1015E0002DEF14F0260EE66E3AEC14F0E552002AC8
:1015F0000050EA6AA00FE96E000EEA22EF500D6E6D
:1016000000500D240D24186E0001FD51185C36E2C7
:10161000060E0DC0DBFF060EDB502FE0F29E8A8C1B
:10162000939A8A8A8A9C8A9A8A8C8A9C8A8A8A8CC9
:101630008A9C8A8C8A9C002A0050EA6AA00FE96E74
:10164000000EEA22EFCF14F0002A0050EA6AA00F41
:10165000E96E000EEA22EFCF13F0100E0D6E143279
:101660001332819AD8B0818A818C819C0D2EF7D754
:101670008A9AF28E060EDB06CED70DD0FE0EE66EEF
:101680003AEC14F0E5520028EA6AA00FE96E000E69
:10169000EA22040EEF6E2DEF14F0270EE66E3AEC00
:1016A00014F0E552040E0024186E0001FD51185C80
:1016B00065E2F29E8A8C939A8A8A8A9C8A8C8A9C9A
:1016C0008A8C8A9C8A8C8A9C002A0050EA6AA00F25
:1016D000E96E000EEA22EFCF14F0002A0050EA6A09
:1016E000A00FE96E000EEA22EFCF13F0100E0D6E80
:1016F00014321332819AD8B0818A818C819C0D2E4C
:10170000F7D78A9A8A8C8A9C8A8C8A9C8A8C8A9C33
:101710008A8C002A0050EA6AA00FE96E000EEA22C5
:10172000EFCF14F0002A0050EA6AA00FE96E000E15
:10173000EA22EFCF13F01350141008E0000000006D
:10174000000000001306000E145AF5D78A9CECC066
:101750000DF00D5009E00000000000000000000046
:10176000000000000D06F5D7100E0D6E0D5004E0C0
:101770008A8C8A9C0D06FAD7F28E0DD0FE0EE66E8C
:101780003AEC14F0E5520028EA6AA00FE96E000E68
:10179000EA22040EEF6E2DEF14F0280EE66E3AECFE
:1017A00014F0E552040E0024186E0001FD51185C7F
:1017B00066E2F29E8A8C939A8A9A8A9C8A8A8A8C9A
:1017C0008A9C8A8C8A9C8A8C8A9C002A0050EA6AAD
:1017D000A00FE96E000EEA22EFCF14F0002A0050AD
:1017E000EA6AA00FE96E000EEA22EFCF13F0100EA6
:1017F0000D6E14321332819AD8B0818A818C819C0B
:101800000D2EF7D78A9A8A8C8A9C8A8C8A9C8A8C1D
:101810008A9C8A8C002A0050EA6AA00FE96E000EAA
:10182000EA22EFCF14F0002A0050EA6AA00FE96E16
:10183000000EEA22EFCF13F01350141008E000005E
:101840000000000000001306000E145AF5D78A9C11
:10185000ECC00DF00D5009E0000000000000000099
:101860000000000000000D06F5D7100E0D6E0D50A3
:1018700004E08A8C8A9C0D06FAD7F28E0DD0FE0EFB
:10188000E66E3AEC14F0E5520028EA6AA00FE96E21
:10189000000EEA22040EEF6E2DEF14F0290EE66E14
:1018A0003AEC14F0E552030E0024186E0001FD51CD
:1018B000185C36E2002A0050EA6AA00FE96E000EBA
:1018C000EA22EFCF13F0F29E8A8C939A040E0D6EEB
:1018D0001332819AD8B0818A818C819C0D2EF8D7E1
:1018E000002A0050EA6AA00FE96E000EEA22EFCF4C
:1018F00014F0002A0050EA6AA00FE96E000EEA22F6
:10190000EFCF13F0100E0D6E14321332819AD8B04F
:10191000818A818C819C0D2EF7D78A9AF28E0DD008
:10192000FE0EE66E3AEC14F0E5520028EA6AA00FCB
:10193000E96E000EEA22040EEF6E2DEF14F02A0E6F
:10194000E66E3AEC14F0E5520028186E0001FD51E5
:10195000185C39E2002A0050EA6AA00FE96E000E16
:10196000EA22EFCF13F0F29E8A8C939A040E0D6E4A
:101970001332819AD8B0818A818C819C0D2EF8D740
:101980008A8C8A9C8A8C8A9C8A8C8A9C8A8C8A9C67
:101990008A8C8A9C8A8C8A9C8A8C8A9C8A8C8A9C57
:1019A000938A080E0D6E818C819CD89081BAD88064
:1019B00013320D2EF8D78A9AF28E13C0E6FF3AEC56
:1019C00014F0E5520DD0FE0EE66E3AEC14F0E5523E
:1019D0000028EA6AA00FE96E000EEA22040EEF6EFC
:1019E0002DEF14F02B0EE66E3AEC14F0E5520028C1
:1019F000186E0001FD51185C42E2002A0050EA6AAC
:101A0000A00FE96E000EEA22EF500D6EFF0E0D5C86
:101A100004E1C66A9368948C31D0800EC76E080EBC
:101A2000C66EC56A0DBCC79EC70E936E8A6A0DB09E
:101A30008A860DB28A880DB48A8A949C8B9C380E53
:101A40000D160D5003E1770EC86E17D0080E0D5C11
:101A500003E13B0EC86E11D0100E0D5C03E1270EA2
:101A6000C86E0BD0180E0D5C03E10E0EC86E05D0CB
:101A7000200E0D5C02E10B0EC86EC68A0DD0FE0E64
:101A8000E66E3AEC14F0E5520028EA6AA00FE96E1F
:101A9000000EEA22040EEF6E2DEF14F02C0EE66E0F
:101AA0003AEC14F0E552030E0024186E0001FD51CB
:101AB000185C01E3BDD0002A0050EA6AA00FE96E6D
:101AC000000EEA22EF500D6E0001010E146E002A86
:101AD0000050EA6AA00FE96E000EEA22EFCF13F081
:101AE000C750040B01E0010E186E1F0EC51418102C
:101AF00001E0F6D7C580C5B0FED70D505DE0FE0E03
:101B000000011314C96EC7B0FED7C750040B01E023
:101B1000010E186E1F0EC514181001E0F6D7C5BCD3
:101B20004AD0002A0050EA6AA00FE96E000EEA22AD
:101B3000EF50C96EC7B0FED7C750040B01E0010ECD
:101B4000186E1F0EC514181001E0F6D7C5BC33D0AF
:101B5000C582C5B2FED7010E00011310C96EC7B011
:101B6000FED7C750040B01E0010E186E1F0EC514FE
:101B7000181001E0F6D7C5BC1ED00001146A0D5044
:101B8000E66E3AEC14F0E5520D5011E0C586C7A0A0
:101B9000FED7C950E66E3AEC14F0E5520D5001083C
:101BA00004E2C59AC588C5B8FED70D06EDD7C58A2B
:101BB000C588C5B8FED725D0010E00011310C96E27
:101BC000C7B0FED7C750040B01E0010E186E1F0E00
:101BD000C514181001E0F6D7C5BC13D00001146A73
:101BE000010EE66E3AEC14F0E552C586C7A0FED7AA
:101BF000C950E66E3AEC14F0E552C58AC588C5B8FE
:101C0000FED7C550400B10E0000114500DE0FD0E52
:101C1000E66E3AEC14F0E5520028EA6AA00FE96E8D
:101C2000000EEA22040EEF6EC584C5B4FED70DD0B7
:101C3000FE0EE66E3AEC14F0E5520028EA6AA00FB8
:101C4000E96E000EEA22040EEF6E2DEF14F02E0E58
:101C5000E66E3AEC14F0E552040E0024186E000112
:101C6000FD51185C01E3ACD0002A0050EA6AA00FD5
:101C7000E96E000EEA22EF500D6E0001010E146EA7
:101C8000002A0050EA6AA00FE96E000EEA22EFCFA8
:101C900013F0C750040B01E0010E186E1F0EC5149F
:101CA000181001E0F6D7C580C5B0FED7FE0E0001C2
:101CB0001314C96EC7B0FED7C750040B01E0010E64
:101CC000186E1F0EC514181001E0F6D7C5BC61D000
:101CD000002A0050EA6AA00FE96E000EEA22EF50D7
:101CE000C96EC7B0FED7C750040B01E0010E186ED5
:101CF0001F0EC514181001E0F6D7C5BC4AD0002A43
:101D00000050EA6AA00FE96E000EEA22EF50C96E99
:101D1000C7B0FED7C750040B01E0010E186E1F0EAE
:101D2000C514181001E0F6D7C5BC33D0C582C5B2C2
:101D3000FED7010E00011310C96EC7B0FED7C75001
:101D4000040B01E0010E186E1F0EC514181001E0FF
:101D5000F6D7C5BC1ED00001146A0D50E66E3AECF1
:101D600014F0E5520D5011E0C586C7A0FED7C9504A
:101D7000E66E3AEC14F0E5520D50010804E2C59A03
:101D8000C588C5B8FED70D06EDD7C58AC588C5B8C4
:101D9000FED7C550400B10E0000114500DE0FD0EC1
:101DA000E66E3AEC14F0E5520028EA6AA00FE96EFC
:101DB000000EEA22040EEF6EC584C5B4FED70DD026
:101DC000FE0EE66E3AEC14F0E5520028EA6AA00F27
:101DD000E96E000EEA22040EEF6E2DEF14F02D0EC8
:101DE000E66E3AEC14F0E552002A0050EA6AA00FC1
:101DF000E96E000EEA22EF500D6E020E00240D2453
:101E0000186E0001FD51185C73E2C750040B01E02D
:101E1000010E186E1F0EC514181001E0F6D7C5800C
:101E2000C5B0FED7002A0050EA6AA00FE96E000E86
:101E3000EA22EF50FE0BC96EC7B0FED7C750040BA5
:101E400001E0010E186E1F0EC514181001E0F6D740
:101E5000C5BC38D0002A0050EA6AA00FE96E000E17
:101E6000EA22EF50C96EC7B0FED7C750040B01E09D
:101E7000010E186E1F0EC514181001E0F6D7C5BC70
:101E800021D00D50E66E3AEC14F0E5520D501AE0F8
:101E9000C550400B17E1002A0050EA6AA00FE96E16
:101EA000000EEA22EF50C96EC7B0FED7C750040B30
:101EB00001E0010E186E1F0EC514181001E0F6D7D0
:101EC0000D06E4D70D5003E1C550400B0DE0FD0EAB
:101ED000E66E3AEC14F0E5520028EA6AA00FE96ECB
:101EE000000EEA22040EEF6EC584C5B4FED70DD0F5
:101EF000FE0EE66E3AEC14F0E5520028EA6AA00FF6
:101F0000E96E000EEA22040EEF6E2DEF14F02F0E94
:101F1000E66E3AEC14F0E5520028186E0001FD510F
:101F2000185C3BE2002A0050EA6AA00FE96E000E3E
:101F3000EA22EF500D6EFF0E0D5C09E19368948C60
:101F4000948E010E066E0001640EEC6F25D0E50E36
:101F5000936E0DA602D08A8201D08A92949C8B9CAB
:101F6000949E0C0E0D140001EC6F030E0D160D5017
:101F700003E1120E066E10D00D0403E1080E066E8A
:101F80000BD0020E0D5C03E1050E066E05D0030EAC
:101F90000D5C02E1020E066E0DD0FE0EE66E3AEC0E
:101FA00014F0E5520028EA6AA00FE96E000EEA225A
:101FB000040EEF6E2DEF14F0300EE66E3AEC14F0D6
:101FC000E5520028186E0001FD51185C23E2002A3A
:101FD0000050EA6AA00FE96E000EEA22EF500D6E83
:101FE0000D50E66E3AEC14F0E5520D5005E1E66A4C
:101FF0003AEC14F0E5520DD093800D500AE0E66AF9
:10200000CEEC14F0E552E66E3AEC14F0E5520D0613
:10201000F4D70DD0FE0EE66E3AEC14F0E55200282F
:10202000EA6AA00FE96E000EEA22040EEF6E2DEFB1
:1020300014F0310EE66E3AEC14F0E552002A00502E
:10204000EA6AA00FE96E000EEA22EF500D6E005012
:102050000D24186E0001FD51185C17E20D50E66E5C
:102060003AEC14F0E552949E0D500EE0002A005018
:10207000EA6AA00FE96E000EEA22EF50E66ECEEC9F
:1020800014F0E5520D06F0D70CD0FE0EE66EF2DB32
:10209000E5520028EA6AA00FE96E000EEA22040E5B
:1020A000EF6EDBD3320EE66EE5DBE552020E002466
:1020B000186E0001FD51185C21E2002A0050EA6A06
:1020C000A00FE96E000EEA22EF508A6E002A00503F
:1020D000EA6AA00FE96E000EEA22EF500D6EC00E04
:1020E0000D14186E3F0E8B1418108B6E380E0D14D5
:1020F000186EC70E89141810896E0CD0FE0EE66E8D
:10210000B9DBE5520028EA6AA00FE96E000EEA2268
:10211000040EEF6EA2D3330EE66EACDBE552030E77
:102120000024186E0001FD51185C63E2002A005083
:10213000EA6AA00FE96E000EEA22EF500D6E002A47
:102140000050EA6AA00FE96E000EEA22EFCF14F009
:10215000002A0050EA6AA00FE96E000EEA22EFCFD3
:1021600013F001500D240D24186E400E185C34E25B
:102170000D50E66E7FDBE5520D502DE0200EE66E31
:10218000CEEC14F0E55214C0E6FFCEEC14F0E552AC
:1021900013C0E6FFCEEC14F0E552E66ACEEC14F084
:1021A000E552E66E67DBE552280EE66EF7DBE55298
:1021B00014C0E6FFF3DBE55213C0E6FFEFDBE552A8
:1021C000E66AECDBE552E66E55DBE552132A000EBB
:1021D00014220D06D1D70CD0FE0EE66E4BDBE55275
:1021E0000028EA6AA00FE96E000EEA22040EEF6EE4
:1021F0000CD0FE0EE66E3EDBE5520028EA6AA00F28
:10220000E96E000EEA22040EEF6E27D3340EE66E5E
:1022100031DBE552002A0050EA6AA00FE96E000E99
:10222000EA22EF500D6E00500D240D24020F186E9F
:102230000001FD51185C4CE20D50E66E1BDBE552CF
:10224000002A0050EA6AA00FE96E000EEA22EFCFE2
:1022500014F0002A0050EA6AA00FE96E000EEA228C
:10226000EFCF13F00D5033E0400EE66E97DBE552F2
:1022700014C0E6FF93DBE55213C0E6FF8FDBE552A7
:10228000002A0050EA6AA00FE96E000EEA22EF5021
:10229000E66E84DBE552480EE66E80DBE55214C044
:1022A000E6FF7CDBE55213C0E6FF78DBE552002A4F
:1022B0000050EA6AA00FE96E000EEA22EF50E66EC7
:1022C0006DDBE552132A000E14220D06CBD70CD07D
:1022D000FE0EE66ECFDAE5520028EA6AA00FE96E3C
:1022E000000EEA22040EEF6EB8D2350EE66EC2DAA8
:1022F000E5520028186E0001FD51185C46E2002AE4
:102300000050EA6AA00FE96E000EEA22EF500D6E4F
:10231000FF0E0D5C05E1BA6ABD6A8A96B16A34D0D7
:1023200094849396B36AB26AC10EB16EBC6ABF6AF6
:102330000D5003E13B0EBE6E21D00D0403E11D0ED6
:10234000BE6E1CD0020E0D5C03E10B0EBE6E16D0ED
:10235000030E0D5C03E1050EBE6E10D0040E0D5C85
:1023600003E1020EBE6E0AD0050E0D5C03E1010E04
:10237000BE6E04D0060E0D5C01E1BE6A010EBB6E9E
:102380000B0EBD6E020EBA6E0CD0FE0EE66E72DA49
:10239000E5520028EA6AA00FE96E000EEA22040E58
:1023A000EF6E5BD2360EE66E65DAE552030E002460
:1023B000186E0001FD51185C35E2F29E939A8A9ADC
:1023C0008A8C8A9C8A8C8A9C8A8C8A9C8A8C8A9C1D
:1023D000002A0050EA6AA00FE96E000EEA22EFCF51
:1023E00014F0002A0050EA6AA00FE96E000EEA22FB
:1023F000EFCF13F0002A0050EA6AA00FE96E000E3A
:10240000EA22EF500E6E180E0D6E143213320E3299
:10241000819AD8B0818A818C819C0D2EF6D78A9AB8
:10242000F28E0CD0FE0EE66E25DAE5520028EA6A3E
:10243000A00FE96E000EEA22040EEF6E0ED2370EE8
:10244000E66E18DAE552F29E939A8A8A8A8C8A9C02
:102450008A9A0D6A0B0E0D5C04E28A8C8A9C0D2A06
:10246000F9D7938A100E0D6E818CD89081BAD880DE
:1024700014321332819C0D2EF7D78A9AF28E14C033
:10248000E6FFF8D9E55213C0E6FFF4D9E552E5D1ED
:10249000380EE66EEFD9E552F29E939A8A9A0D6A4B
:1024A0001C0E0D5C04E28A8C8A9C0D2AF9D7F28EF0
:1024B000D4D1390EE66EDED9E552002A0050EA6A20
:1024C000A00FE96E000EEA22EF500D6E00500D24B1
:1024D0000D24186E0001FD51185C2CE2F29E939AB7
:1024E000070E0DC0DBFF070EDB5020E0002A005076
:1024F000EA6AA00FE96E000EEA22EFCF14F0002A7C
:102500000050EA6AA00FE96E000EEA22EFCF13F046
:10251000100E0D6E13361436819AD8B0818A818CD4
:10252000819C0D2EF7D7070EDB06DDD78A9A938A9A
:10253000F28E0CD0FE0EE66E9DD9E5520028EA6AB6
:10254000A00FE96E000EEA22040EEF6E86D13A0E5D
:10255000E66E90D9E552002A0050EA6AA00FE96EB3
:10256000000EEA22EF500D6E0001FD51005C2BE2DF
:1025700001500D240D24186E400E185C24E20D50FD
:10258000E66E78D9E552F29E938A080E0DC0DBFF05
:10259000080EDB5016E0100E0D6E818CD89081BABB
:1025A000D88013361436819C0D2EF7D714C0E6FF61
:1025B00061D9E55213C0E6FF5DD9E552080EDB068E
:1025C000E7D7F28E0CD0FE0EE66E54D9E552002805
:1025D000EA6AA00FE96E000EEA22040EEF6E3DD10A
:1025E0003B0EE66E47D9E552C50E936E8A6A949EFD
:1025F00034D13C0EE66E3ED9E552002A0050EA6A1C
:10260000A00FE96E000EEA22EF500D6E0D040024BB
:10261000E8380F0B186E0001FD51185C21E2F29EA4
:102620000E6A0D5000081AE20E500BE1002A00500D
:10263000EA6AA00FE96E000EEA22EFCF13F0080E4F
:102640000E6E1336829ED8B0828E8182000000000A
:102650000000000081920D060E06E3D7F28E0CD02A
:10266000FE0EE66E07D9E5520028EA6AA00FE96E71
:10267000000EEA22040EEF6EF0D03D0EE66EFAD8A0
:10268000E5520028186E0001FD51185C34E20D047B
:102690000124E8380F0B196E400E195C2CE2002A59
:1026A0000050EA6AA00FE96E000EEA22EF500D6EAC
:1026B0000D50E66EDFD8E552F29E080E0E6E0D50FC
:1026C000000817E2818200000000000000008192F3
:1026D000D89081B0D88013360E060E5002E00D045B
:1026E00006E1080E0E6E13C0E6FFC4D8E5520D06D3
:1026F000E6D7F28E0CD0FE0EE66EBCD8E55200286E
:10270000EA6AA00FE96E000EEA22040EEF6EA5D071
:10271000400E015C09E20150EA6A600FE96E000EAA
:10272000EA22EF6A012AF4D7016A04010CBF0BD038
:10273000400EE66E600EE66E000EE66E06EC15F0DC
:10274000E552E552E552006888D0F00EE66E92D868
:10275000E552020E0024186E0001FD51185C25E2BE
:10276000002A0050EA6AA00FE96E000EEA22EFCFBD
:1027700014F0002A0050EA6AA00FE96E000EEA2267
:10278000EFCF13F014C0E6FF75D8E55213C0E6FF93
:1027900071D8E55214C0EAFF13C0E9FFEF500D6E87
:1027A0000D50E66E67D8E5520CD0FE0EE66E62D88C
:1027B000E5520028EA6AA00FE96E000EEA22040E34
:1027C000EF6E4BD0F10EE66E55D8E552030E0024A5
:1027D000186E0001FD51185C2EE2002A0050EA6AD2
:1027E000A00FE96E000EEA22EFCF14F0002A00508D
:1027F000EA6AA00FE96E000EEA22EFCF13F0002A7A
:102800000050EA6AA00FE96E000EEA22EF500D6E4A
:1028100014C0E6FF2FD8E55213C0E6FF2BD8E552CF
:102820000D50E66E27D8E55214C0EAFF13C0E9FF49
:102830000D50EF6E0CD0FE0EE66E1CD8E55200284F
:10284000EA6AA00FE96E000EEA22040EEF6E05D0D0
:10285000FE0EE66E0FD8E55200D0002A01D0899214
:10286000090EE15C02E2E16AE552E16EE552E7CF72
:10287000D9FF1200D9CFE6FFE1CFD9FF0001EA511D
:102880000AE00A0E025C11E20250022AEA6AE00F34
:10289000E96E000E06D00150012AEA6A600FE96E67
:1028A000000EEA22FE0EDBCFEFFF400E015C13E1CB
:1028B000016A04010CBF0CD0400EE66E600EE66E9D
:1028C000000EE66E06EC15F0E552E552E55203D037
:1028D0000001010EEA6FE552E7CFD9FF1200D8CF11
:1028E000E4FFE0CFE4FFE46EDACFE4FFE2CFDAFF0B
:1028F000F3CFE4FFF4CFE4FFE652C2B2FED79E9CD2
:1029000007C009F008C00AF0C4CF08F0C3CF07F031
:102910000B50075E0C50085AE10E0902F4CF10F07C
:10292000F3CF0FF0E10E0A02F35010260F500326EA
:1029300010500422E40E0702F4CF10F0F3CF0FF092
:10294000E40E0802F35010260F50035E1050045A94
:102950000001043402E3036A046A05500001D880D0
:10296000045402E205C004F004C0BEFF000103509D
:10297000E840E8403F0B300B1E6ECF0EBD141E101A
:10298000BD6EE552E5CFF4FFE5CFF3FFE5CFDAFF0B
:10299000E550E5CFE0FFE5CFD8FF1000D9CFE6FF47
:1029A000E1CFD9FFF29EFE0EDB50156EECC00FF0AA
:1029B000080E0E6E0FB404D015AE829E15BE828E28
:1029C0000650176E172EFED70FA681820FB6819282
:1029D0000FA405D015AE829E15BE828E02D0813026
:1029E00015360650176E172EFED70FA681920FB61A
:1029F00081820FA402D0813015360E2EDBD7F28EE5
:0C2A0000155000D0E552E7CFD9FF1200BE
:042A0C00D9CFE6FF39
:102A1000E1CFD9FFE65204010CAF02D0000E33D053
:102A2000FC0EDB50400805E2400EF36EFC0EF3CFC7
:102A3000DBFFDF6AFC0EDB50DF5C19E2DF50E76E84
:102A4000FD0EDBCFE9FFFE0EDBCFEAFFE750E92604
:102A5000000EEA22EF50E66EDF50EA6A580FE96E88
:102A6000050EEA22E552E750EF6EDF2AE3D7FC0EAF
:102A7000DBCF0DF404010CAD02D0880E01D0C80EDE
:102A80000C6FFC0EDB50E552E552E7CFD9FF120088
:102A9000D9CFE6FFE1CFD9FF0101136B040108BFD5
:102AA00032D0FC0EDBCF18F00951D880185403E265
:102AB000FC0E09C4DBFF0101136BFC0EDB50135D40
:102AC00019E21351EA6A180FE96E050EEA22EF5077
:102AD000E66E1351E76EFD0EDBCFE9FFFE0EDBCF96
:102AE000EAFFE750E926000EEA22E552E750EF6ED2
:102AF000132BE3D70401400E096F08AD02D0880EF6
:102B000001D0C80E086F01011351E552E7CFD9FF7C
:102B100012000101136B1E0E716E0401400E096F4D
:102B2000180E186E050E18C00AF40B6F880E086F89
:102B3000580E186E050E18C00EF40F6F400E0C6F75
:102B40001200D9CFE6FFE1CFD9FFE65202C5DFFF81
:102B50000101010E076FE552E552E7CFD9FF1200E0
:102B6000D9CFE6FFE1CFD9FFE65202C5DFFF010171
:102B7000010E076FE552E552E7CFD9FF1200D9CF1A
:102B8000E6FFE1CFD9FF020EE1261F0E0501001579
:102B9000010865E1045163E101C5DFFF060EDF5C5A
:102BA00023E1010E03C5DBFFDB50210809E1010130
:102BB000010E076FD50E0A6F330E0B6F090E0CD086
:102BC000010EDB5022080DE10101010E076FF50E29
:102BD0000A6F330E0B6F220E0E6F0F6B010E106F0C
:102BE00003D0010EDB502308600E050100152008FC
:102BF00036E1DF0402E1A5DF32D0090EDF5C05E13A
:102C00000101010E066FACDF2AD0020EDF5C07E186
:102C10000101010E076F110E086F010E12D00A0E8E
:102C2000DF5C06E10101010E076F03C511F117D04A
:102C3000030EDF5C0CE10101010E076F120E086F3D
:102C4000010E096F010E0E6F0F6B106B08D00B0E8B
:102C5000DF5C05E10101010E076F02C512F1020EF2
:102C6000E15C02E2E16AE552E16EE552E7CFD9FFAD
:102C70001200D9CFE6FFE1CFD9FF020EE126800E88
:102C80000501005D3CE103C5DFFF010E02C5DBFF6E
:102C9000DF0409E10101010E076FBA0E0A6F330E5E
:102CA0000B6F120E28D0020EDF5C09E10101010E4C
:102CB000076FCC0E0A6F330E0B6F290E1CD0030E5C
:102CC000DF5C1DE10101010E076FDB5004E1170E0F
:102CD0000A6F340E0AD0010EDB0404E11B0E0A6FEA
:102CE000340E03D03B0E0A6F340E0B6F0AC1F6FF91
:102CF000F76E0800F5500E6F0F6B010E106F020E8D
:102D0000E15C02E2E16AE552E16EE552E7CFD9FF0C
:102D10001200D9CFE6FFE1CFD9FF030EE1261F0E47
:102D200005010015DF6E106B116BDF500DE1010125
:102D3000010E076F035102E00501108101010151ED
:102D400035E00501108332D0DF0404E10101010EFA
:102D5000076F2CD0020EDF5C29E10F0E0415E76E21
:102D6000010EE7CFDBFF800E0415E76E020EE7CF02
:102D7000DBFF0101010E076FDB50080DF3500C6FF4
:102D80000D6B000E0C27040E0D23020EDB5004E029
:102D9000040E0C27000E0D230CC1E9FF0DC1EAFF44
:102DA000EF50040B03E00501010E106F0101075104
:102DB00008E0100E086F050E096F020E0E6F0F6B04
:102DC000106B030EE15C02E2E16AE552E16EE5524E
:102DD000E7CFD9FF1200D9CFE6FFE1CFD9FF040E2C
:102DE000E1261F0E05010015DF6E010E02C5DBFF97
:102DF000DF5011E1010EDB044CE10101010E076F10
:102E0000030E0501015D04E10101010E016F41D0D6
:102E10000101016B3ED0020EDF5C3BE10F0E041599
:102E2000E76E020EE7CFDBFF800E0415E76E030EA0
:102E3000E7CFDBFF010EDB502CE1020EDB5029E077
:102E40000101010E076F020EDB50080DF3500C6FED
:102E50000D6B000E0C27040E0D23030EDB5004E057
:102E6000040E0C27000E0D23030E0501015D02E187
:102E7000840E0AD0030EDB0406E10CC1E9FF0DC18C
:102E8000EAFFEF6A06D0880E0CC1E9FF0DC1EAFF28
:102E9000EF6E040EE15C02E2E16AE552E16EE5529A
:102EA000E7CFD9FF1200D9CFE6FFE1CFD9FFE65235
:102EB00001C5DFFF600E0501001554E1050EDF5C62
:102EC00008E10101010E076F040E006F02C502F157
:102ED00049D0060EDF5C02E1CCDE44D0090EDF5C97
:102EE0000EE10101010E076F02C504F1045103E177
:102EF000040E006F37D0050E006F0BDE33D0080EC6
:102F0000DF5C07E10101010E076F040E086F010E7F
:102F100017D0DF5002E1FDDE25D0DF0403E0030E11
:102F2000DF5C02E158DF1ED00A0EDF5C0FE1010119
:102F3000010E076F0501106B0101100E086F050EE1
:102F4000096F010E0E6F0F6B106B0CD00B0EDF5C58
:102F500004E10101010E076F05D0070EDF5C02E0FE
:102F60000C0EDF5CE552E552E7CFD9FF1200D9CF56
:102F7000E6FFE1CFD9FF030EE1260101080E0E5D49
:102F8000000E0F5907E2010E0EC1DBFF020E0FC14A
:102F9000DBFF07D0080EF36E010EF3CFDBFF020E4E
:102FA000DB6AFC0E04010417010E020EDBCF19F0E0
:102FB000000E030E191619C018F019500413FF0E55
:102FC000E76E010EDBCF18F0020EE750181618C09E
:102FD00005F4100E186E050E1B6A18C006F4076F74
:102FE000010EDB5001010E5F020EDB500F5B100E75
:102FF0000C6F050E0D6F100524E1DF6ADFCF18F0AE
:10300000010EDBCF19F0020EDBCF1AF01950185C5D
:10301000000E1A5439E20AC1F6FF0BC1F7FF0A2B62
:10302000000E0B230800F550E66E0CC1E9FF0DC140
:10303000EAFF0C2B000E0D23E552E750EF6EDF2A5E
:10304000DDD7DF6ADFCF18F0010EDBCF19F0020EFB
:10305000DBCF1AF01950185C000E1A5415E208C1A3
:10306000E9FF09C1EAFF082B000E0923EF50E66EC5
:103070000CC1E9FF0DC1EAFF0C2B000E0D23E55238
:10308000E750EF6EDF2ADED7030EE15C02E2E16A71
:10309000E552E16EE552E7CFD9FF1200D9CFE6FF46
:1030A000E1CFD9FF040EE1260401F3500111E66ED1
:1030B000D950020FE96EDACFEAFFE552E750EE6E23
:1030C000ED6A020EDB5001010E27030EDB500F23C9
:1030D000100E086F050E096FDE6ADD6ADECF18F08C
:1030E000DDCF19F0020EDBCF1AF0030EDBCF1BF0A1
:1030F0001A50185C1B50195818E208C1E9FF09C1A1
:10310000EAFF082B000E0923EF50E66E0CC1E9FF21
:103110000DC1EAFF0C2B000E0D23E552E750EF6EB8
:10312000DF2A010EDBE3DB2AD9D7040EE15C02E2E1
:10313000E16AE552E16EE552E7CFD9FF12000401E2
:10314000049F009F0101056B076B066B0E6B0F6BF5
:10315000AADE15DD010107510EE10401080E016F21
:10316000000E186E050E1A6A1B6A18C002F4036F6F
:10317000840E006F30D0050100AF2FD001010E5139
:103180000501065D01010F510501075904E206C55D
:103190000EF107C50FF1EBDE0101020E056F040110
:1031A000080E016F000E186E050E196E1A6A1B6A62
:1031B0001A6A1B6A18C002F4036F800E006F100EAB
:1031C000186E050E196E1A6A1B6A1A6A1B6A18C0F5
:1031D00006F4076FC80E046F16D00101010E056FCB
:1031E0000401056BC80E046F080E016F100E186EF7
:1031F000050E196E1A6A1B6A1A6A1B6A18C002F455
:10320000036FC80E006F6D9812000101056B040179
:10321000080E016F000E186E050E18C002F4036F41
:10322000880E006F046B1200D9CFE6FFE1CFD9FF03
:10323000020EE1266C5024E13C0E04010015E8402A
:10324000E8403F0BDF6E0D0EDF5C02E178DF35D02A
:103250000101050531E122DF0101065109E0010EFE
:1032600002C5DBFF020E0501035D02E0030E035DF4
:10327000040100AD02D0880E01D0C80E006F1DD031
:10328000040E6C5C1AE16E500AE1040E0101005D4F
:1032900006E102C56EFF6E5002E1030E006F020EE2
:1032A0000101055D09E163DE040104AD02D0880E71
:1032B00001D0C80E046F01D0A8DF020EE15C02E26B
:1032C000E16AE552E16EE552E7CFD9FF12006DB633
:1032D00006D06D6A696A6D860101010E006F0101F9
:1032E000000509E16D50200B06E1686A696A698092
:1032F0006988020E006F12006D9269946894120042
:10330000689C120070A002D080DF7090689A120052
:1033100012006A6A686A9F0E6B6E7B0E696E6E6A37
:10332000160E706E68A602D06896FCD76D986DDF99
:103330000101016B036B046B030E006F12000101AE
:10334000005101E112006850040B04E06950040BC5
:1033500001E0D2DF6DB212006850010B04E0695049
:10336000010B01E0D6DF6850100B04E06950100B30
:1033700001E0CEDF6850400B04E06950400B01E0F3
:10338000BFDF6850200B04E06950200B01E0BADF7A
:103390006850020B04E06950020B01E06892030ED2
:1033A0000101005D01E212006850080B05E0695060
:0A33B000080B02E039DF68961200F6
:0633BA00120100020000F8
:1033C0000008D804000101000102000109022900DF
:1033D000010100A0320904000002030000000921DD
:1033E00001010001222200070581034000010705B9
:1033F000010340000106A0FF0901A1010903150016
:1034000026FF007508954081020904150026FF007B
:10341000750895409102C00403090420034F007011
:103420000065006E002000500072006F006700729F
:103430000061006D006D00650072003E034F00707A
:103440000065006E002000500072006F006700727F
:103450000061006D006D00650072002000200055C5
:10346000005300420020004800490044002000634F
:09347000006C00610073007300A0
:013479000052
:06347A002A0EF66E000EA2
:10348000F76E000EF86E00010900F550F86F0900A4
:10349000F550F96F03E1F86701D03DD00900F55010
:1034A000F36F0900F550F46F0900F550F56F09004E
:1034B0000900F550E96E0900F550EA6E09000900AF
:1034C0000900F550F66F0900F550F76F0900090083
:1034D000F6CFFAF0F7CFFBF0F8CFFCF0F3C0F6FF31
:1034E000F4C0F7FFF5C0F8FF0001F65302E1F7530F
:1034F00007E00900F550EE6EF607F8E2F707F9D796
:10350000FAC0F6FFFBC0F7FFFCC0F8FF0001F807A8
:08351000000EF95BBFD71200A9
:083518000F0EC112140E6F6EBC
:103520000101006B0101016B0101046B22EC00F051
:1035300067EC19F06FBE02D09FEC19F062EC00F05E
:02354000F7D7BB
:0E35420013EE00F023EE00F0F86A1D9C3DEC45
:0E3550001AF0B6EC1AF08CEC1AF0FBD7120051
:02355E0000EE7D
:0C35600000F00F0EEE6AEA62FDD71200C8
:02356C0012004B
:02356E0000005B
:10357000000000640100000000AB03000000000038
:0635800000000000000045
:020000040030CA
:0100000022DD
:010001000EF0
:010002003DC0
:010003001EDE
:0100050000FA
:010006008178
:0200000400F00A
:100000004F70656E2050726F6772616D6D65722002
:10001000762E20302E362E31202D20436F707972AF
:100020006967687420284329203230303920416CB8
:10003000626572746F204D616363696F6E69202D14
:100040002054686973206973206672656520736F38
:070050006674776172650020
:00000001FF
